:1000000033C0000044C0000042C0000040C00000F7
:100010003EC000003CC000003AC0000038C00000F4
:1000200036C0000034C0000032C0000030C0000004
:100030002EC000002CC000002AC0000028C0000014
:1000400026C0000024C0000022C0000020C0000024
:100050001EC000001CC000001AC0000018C0000034
:1000600016C0000014C0000011241FBECFEFD4E062
:10007000DEBFCDBF11E0A0E0B1E0E2E2FDE002C0F2
:1000800005900D92A230B107D9F733D548C6B8CF45
:10009000BF92CF92DF921F93CF93DF93DC01CB010E
:1000A000142FE901E4E3FCE10F921F927EEF6AE96D
:1000B00056E543E8D92EC82EBA2E212F1D2E0C2E20
:1000C00009952131F9F71F900F90DF91CF911F9182
:1000D000DF90CF90BF900895BF92CF92DF921F9391
:1000E000CF93DF93DC01CB01142FE901E4E3FFE1BF
:1000F0000F921F927EEF6AE956E543E8D92EC82E8B
:10010000BA2E212F1D2E0C2E09952131F9F71F90A3
:100110000F90DF91CF911F91DF90CF90BF90089506
:10012000CF93DF93FA01E9012138310510F0C0E8DF
:10013000D0E0AB01BC0140789E01CF01D1D4CE010B
:10014000DF91CF9108952F923F924F925F926F92DD
:100150007F928F929F92AF92BF92CF92DF92EF9257
:10016000FF920F931F93CF93DF934A01E901213848
:10017000310510F0C0E8D0E01E01369427946B01E1
:100180007C0120E8C222D40180E090E060E070E0D1
:1001900082159305B9F0F601E819F909EA0FFB1F7A
:1001A000259134914D915D912417350709F071E047
:1001B00040955095422B532B4F3F5F4F09F061E024
:1001C0000196E6CF772351F1662339F020E030E045
:1001D00043E0C701B601F801099526013701A12CBA
:1001E000B12CA214B30491F0F401219131914F018B
:1001F00041E0C301B201F8010995F2E04F0E511C34
:10020000611C711C2FEFA21AB20AEBCF20E030E084
:1002100045E0C701B601F801099502C0C0E0D0E091
:10022000CE01DF91CF911F910F91FF90EF90DF9062
:10023000CF90BF90AF909F908F907F906F905F9086
:100240004F903F902F9008950F931F93682F70E069
:1002500080E090E048E08B019C013695279517954A
:10026000079560FF0BC0C901B80150E2652753E84C
:10027000752758EB85275DEE952702C0C901B801A7
:10028000415049F71F910F910895CF92DF92EF925D
:10029000FF92C72ED82EE92EFF24842F8627D4DF85
:1002A0006C257D258E259F25FF90EF90DF90CF90C8
:1002B000089528E088E190E00FB6F894A89580931F
:1002C00060000FBE20936000A895F894D4E0CEEFB4
:1002D0002CE1299320E0299314BEFFCF8FEF0895DE
:1002E00084C00000C3C00000A7C00000A5C000007B
:1002F000A3C00000A1C000009FC000009DC000007E
:100300009BC0000099C0000097C0000095C000008D
:1003100093C0000091C000008FC000008DC000009D
:100320008BC0000089C0000087C0000085C00000AD
:1003300083C0000081C000007FC000007DC00000BD
:100340007BC0000079C000007E3FF9F76A39F9F7F9
:100350005635F9F74338F9F7EC2DFD2DB7B6B0FC5B
:10036000FDCF27BFE895B7B6B0FCFDCF21E1B7B60A
:10037000B6FCF4CF08955553422076302E39372EEF
:10038000312C206279205374657068616E2042615F
:100390006572776F6C66000009021200010100802F
:1003A0003209040000000000000012011001FF00EB
:1003B0000008C016DC050201010200010E03550011
:1003C000530042006100730070001C037700770047
:1003D00077002E00660069007300630068006C00FF
:1003E0002E00640065000403090411241FBECFEF32
:1003F000D4E0DEBFCDBF24B7D4E0CEEF39913C319D
:10040000399109F03FEF30933D0120933C0111E019
:10041000A0E0B1E0EAEFFFE302C005900D92A63044
:10042000B107D9F721E0A6E0B1E001C01D92AC33DD
:10043000B207E1F749D14FC353CFA82FB92F80E0BE
:1004400090E041E050EA609530E009C02D918227AC
:100450009795879510F084279527305EC8F36F5FD6
:10046000A8F30895EADF8D939D930895CF93CFB7B6
:10047000CF93DF93C3954F9BE9F74F9B0BC04F9BE7
:1004800009C04F9B07C04F9B05C04F9B03C04F9BAC
:1004900001C089C06F93C0911F01DD27CA5DDE4F87
:1004A0002F9365E54F9B03C02F916F91E6CF0F937C
:1004B0001F934F9320E040E15F9309B1047807FB5D
:1004C00027F93F9350E03BE039C0147840642F7720
:1004D000012F5F5F1EC0406819B114782F7752500A
:1004E0001FC0406409B12F770478D1F15F5F00C06D
:1004F00023C0406219B12F77147891F15F5F00C07B
:1005000025C004781027515012F45D5F000011508F
:1005100027952C3F19B1C8F614780127015027956B
:100520002C3FC8F64227499309B1047810274F732E
:10053000115027952C3FA8F64695469519B1147889
:1005400079F00127015027952C3F98F66B5A60F3FC
:10055000315009B1B0F600C011E01CBB002717C034
:100560003B503195C31BD04011E01CBB0881033CBC
:10057000F9F00B34E9F020911D011981110F1213CC
:10058000EDCF093651F10D3211F0013E39F70093EC
:1005900024013F915F914F911F910F912F916F9186
:1005A000CCB3C0FD67CFDF91CF91CFBFCF9118956E
:1005B00020912401222369F310912201112339F59E
:1005C00034303AF13093220120931E0110911F0123
:1005D0003BE0311B30931F011CC000912201013010
:1005E000B4F40AE53091010134FD14C00093010117
:1005F000C2E1D1E013C0052710E000C000000BB934
:100600001AC0052710E0221F1DC010E021C04AE5D6
:1006100002C032ED432FC4E1D0E032E01AB11468D9
:100620005F9A0BB11AB954E820E865E320FF05276B
:100630000BB9279517951C3FF0F66695B8F7B1F7FB
:1006400020FF05270BB9279517951C3FD0F6279556
:10065000179517FF052700001C3F0BB9B0F629912D
:100660003A9519F70B7710912301110FC651D0401D
:100670000BB911F010931D0111E01CBB00681AB1F9
:100680001B77402F4B7754E05A95F1F70BB91AB905
:100690004BB97FCFFC01938184812281203339F4CF
:1006A0008370E82FF0E0EE5FFE4F80810895203ADE
:1006B00009F4FBC1203C19F46581FFD103C02F3F31
:1006C00009F411EF80E008951AB880E48BB981E055
:1006D00085BF82E085BF83E0A89531978040E1F730
:1006E00080913C01877F21F480913D01882381F036
:1006F0004E9B0EC0F894579A1BB81DBA1092690011
:1007000081E085BF15BEE0910A01F0910B010995CA
:100710001EEF14BE88E10FB6F8948093600010922B
:1007200060000FBE80916900826080936900E89A42
:10073000579A8DE0A89531978040E1F757987894C3
:1007400000912201035007FD2BC180911F01CCE0D5
:10075000D0E0C81BD109CA5DDE4F80911E018D32E9
:1007600009F0B5C0083009F019C183EC809312017B
:100770008AE580930101109211014881842F8076CF
:100780003981882399F186E091E09093210180934B
:100790002001333031F4CE017DDF8093090124E064
:1007A0008CC03530F9F03A30E9F08CEF830F8630A9
:1007B00098F48A819B819093100180930F013930C6
:1007C00099F08E8180930E018D81827080930D014E
:1007D00030930C012FEF6BC0323011F41E7F04C038
:1007E000116002C021E069C020E067C08A811092D8
:1007F0001B01311106C010921C018BE191E022E037
:1008000050C0353019F4809323013DC03630A9F52E
:100810009B81913019F48AEC98E304C0923041F442
:1008200088EB98E3909321018093200122E121C07D
:100830009330F1F4811108C086E099E3909321018F
:100840008093200124E015C0813041F48AEE98E3C2
:1008500090932101809320012CE10BC0823041F460
:100860008CED98E390932101809320012EE001C04C
:1008700020E080E48093110118C0383079F03930DD
:1008800031F4809325018BE191E020E00AC021E062
:100890003A3009F020E08BE191E003C085E291E07D
:1008A00021E090932101809320012F3F31F447FDF7
:1008B0002E8180E88093110107C08F81811104C0CF
:1008C0008E81821708F4282F2093000167C0809141
:1008D000110187FF63C080910E01801708F4082F73
:1008E000801B80930E01DD24D3948111D12C809143
:1008F0000C018730C0F0CC2EEC2EFD2E8E2D8C19E5
:10090000801708F048C0D7016D917D0180910F01DB
:10091000909110019C012F5F3F4F30931001209365
:100920000F01CBD0EBCF80910D01E0910F01F09141
:100930001001DE0100FD0395025048F1F83338F54F
:1009400022D0F8940D901D9021E017D02E2F2E5F0D
:100950002F7731F0DD2079F0882369F0003059F4E9
:1009600023E00BD010D025E008D00DD007B606FE4E
:1009700002C021E102D03296DFCFF89427BFE8957C
:1009800011247894089507B600FCFDCF0895F093E4
:100990001001E0930F01D11010920001109222017A
:1009A0008091010184FF6BC0809100018F3F09F4A9
:1009B00066C0082F893008F008E0801B8093000192
:1009C0008091120198E8892780931201002309F48D
:1009D0004AC08091110187FF28C080910E018017C5
:1009E00008F4082F801B80930E01D0900C01C3E106
:1009F000D1E083E191E02C2F281B2017A0F5E09097
:100A00000F01F0901001B6E0BD1518F4C7014DD0EC
:100A100002C0F701849188832196FFEFEF1AFF0A45
:100A2000F0921001E0920F01E4CFE0912001F091EB
:100A3000210186FF0BC083E191E0DC0124912D931D
:100A40003196202F280F2A13F9CF09C083E191E0B6
:100A5000DC0121912D93202F280F2A13FACFF09338
:100A60002101E0932001602F83E191E0FBDC0C5F2A
:100A70000C3019F08FEF809300010093010184E1A5
:100A800099B1947831F48150D9F7109223011092E2
:100A90001D01103118F04E99105104C0123010F0A1
:100AA0004E9B125011114CCE25CEF999FECF92BD1E
:100AB00081BDF89A992780B50895262FF999FECF20
:100AC0001FBA92BD81BD20BD0FB6F894FA9AF99A6B
:100AD0000FBE01960895F894FFCFFF5A1E940600AA
:100AE000FA01DC0102C005900D9221503040D8F788
:100AF0000895CF93DF93CDB7DEB7C058D1090FB6B5
:100B0000F894DEBF0FBECDBF84B714BE98E10FB618
:100B1000F89490936000109260000FBE579AF8947A
:100B200056985E9A209A219A559A539A5D9A83FD17
:100B3000ECC0C0900001D0900101E12CF12C6FEFCE
:100B40007FEFCB01F701EC0DFD1D44919EDB2FEFF4
:100B5000E21AF20AE114E8E0FE06A1F76632704EEE
:100B600080429E4409F0ADC0198280E090E0F60119
:100B7000E80FF91F45915491FC01F85C25913491DF
:100B80004217530719F081E0898305C00296811549
:100B900028E0920761F78981882309F492C018E65A
:100BA000C12E18E3D12EE12CF12CB701A60140781B
:100BB00020E830E0CE01019693DFC701B601685608
:100BC0007A4F8F4F9F4F08E410E020E830E0AE01ED
:100BD0004F5F5F4FB8DA80E8C80ED11CE11CF11CF2
:100BE000E8E6CE16EAE3DE06E104F104F1F6C12CF4
:100BF000B8E3DB2EE12CF12C5601F8E3BF1A40E8F4
:100C000050E06FEF70E0CE01019682D0409100017C
:100C1000509101014A0D5B1D662757FD6095762FA7
:100C200020E830E0CE0101965BDF0CE610E020E822
:100C300030E0AE014F5F5F4FC701B60184DA20E8B4
:100C4000C20ED11CE11CF11CC1148BE3D806E104D7
:100C5000F10491F6E12CA8E0FA2EEA18FB0840E82E
:100C600050E06FEF70E0CE01019652D09701E1E8BD
:100C7000EE16F10410F020E830E0409100015091B0
:100C800001014A0D5B1D662757FD6095762FCE0149
:100C9000019626DFB501785C80E090E008E410E082
:100CA00020E830E0AE014F5F5F4F4DDAF0E8AF0E65
:100CB000B11C20E8E21AF108A11488E0B80678F225
:100CC000299A289A20E630E0C901880F991F820FDF
:100CD000931F0596009779F0EFE9FFE03197F1F760
:100CE00000C000004E9905C05B984E9BFECF20E6E9
:100CF00030E00197EFCF8BB198E089278BB9215075
:100D000031092115310501F7D4DA5B9AA895FECF98
:100D1000DC0101C06D9341505040E0F70895F89414
:020D2000FFCF03
:020D2200E002ED
:00000001FF
